S12310008639B7FCF48E0FF0CE13C4BD1530CE3030FF156AFF156D7F03097F030ABD1356C8
S1231020B6FCF44724F7B6FCF5CE0105FF03027F0304BD10A57F03077F03087F03057F0311
S123104006BD10E0CE154BBD1530BD1207BD115CBD1223BD11B6CE123FBD1530BD1207BD7F
S1231060115CBD1231F603042705B701042003BD11B6860ABD1576860DBD15767C0304B687
S12310800304810226C4B6030681162608860CB703067A030781152654CE12E2BD15307C2E
S12310A0030A7E102F7D030927087F0309CE156D8D0E7D030A27087F030ACE156A8D0139DB
S12310C0A601E600840FC40F585858581B8B011916C40FCB30E701444444448B30A7003982
S12310E04FCE00000826FD4C811426F539B6030581162608860CB703057A03088115261842
S1231100CE133BBD1530B60104BD11B6CE130BBD15307C03097E102FCE12A2BD1530BD15E5
S123112073813127037E1141BD1207CE133BBD1530B60104BD11B6860ABD1576860DBD151C
S123114076B6030581102227CE12AFBD1530BD1207BD115CBD1231BD11B620E516C40F5C1E
S1231160C1012705C10A220439C60B39C60A398115221EB10306220D2731CE12C4BD153083
S12311807C030A2009CE12D1BD15307C03097E102FB60308270D7A0308B60305800AB70325
S12311A005209ECE12A7BD153020CFCE1333BD153020DB7E102F36840F161B1B1B1B5FCEAA
S12311C01241FF0300BB0301F90300B70301F70300FE0300C6058D25862FBD1576328430E5
S12311E044CE12825FFF0300BB0301F90300B70301F70300FE0300C608BD11FD39A600BD3E
S12312001576085A26F739FE03028C0139260BCE14FCBD153031317E101DFE0302A6007C7B
S1231220030339C10B26037C0307FB0306F7030639C10B26037C0308FB0305F703053920DC
S1231240042020414345202054574F544852454520464F555220464956452020534958539E
S12312604556454E4549474854204E494E45202054454E204A41434B515545454E204B49EF
S12312804E4753504144455320204845415254532020434C5542532020204449414D4F4E1D
S12312A044530A0D3F1A040A0D0742555354040A0D4445414C4552204452415753204120D9
S12312C0202020040A0D07594F552057494E0A0D040A0D074445414C45522057494E530A2C
S12312E00D040A0D42204C20412043204B204A20412043204B2020202059204F205520204F
S123130020572049204E20212021040A0D42204C20412043204B204A20412043204B202028
S123132020204920202020572049204E202120212021040A0D0750555348040A0D4D59206C
S1231340444F574E204341524420574153202004CE14FCBD1530BD153DBD1365BD138EBD89
S123136013A724F539B60103BA0102BA0101BA01002603730103B60103444444B801034746
S12313804776010076010176010276010339B60100B80101B80102B8010316840F810C2F9A
S12313A002800DC4301B39CE0105E6002B0B11270A088C0139270B20F1A7008C013827027A
S12313C00C390D3906060C00000000000A0D54484953204953204D4F544F524F4C4120426C
S12313E04C41434B4A41434B2E2E2E2E2E2E2E2E2E2E2E2E2E2E2E54525920594F55522075
S12314004C55434B2E2E2E2E2E210D0A06074445414C4552204D55535420484954204F4E96
S1231420203136204F52204C45535320414E44205354414E44204F4E2031372E0D0A0000F2
S12314400000004143455320434F554E542031204F52203131202C204641434520434152BE
S1231460445320434F554E542054454E2E0D0A0000000000424C41434B4A41434B205749A6
S123148054482041434520414E44204120464143452043415244204F522054454E0D0A0027
S12314A0000000005449455320434F554E5420415320412050555348204E4F2057494E4EBC
S12314C045522E0D0A0000000000445552494E4720504C41592054595045203120464F5253
S12314E02041204849542C3020544F205354414E44205041540D0A00000000000D0A06028E
S1231500000053485546464C45204E4F5720494E2050524F47524553532E2E2E2E2E2E2E18
S12315202E2E2E2E2E2E06010D0A000000000004A6008104260139BD15760820F3CE0105AF
S123154086FFA700088C013926F8390C0000000D0A00000000000D504C41594552094445A7
S10D1560414C45520D0A0808080624
S104156C0971
S10D156F0D0A0A047EC0067EC003C4
S9030000FC
